:020000041000EA
:1000000000B5324B212058609868022188439860DF
:10001000D860186158612E4B002199600221596106
:100020000121F02299502B49196001219960352056
:1000300000F044F80222904214D00621196600F024
:1000400034F8196E01211966002018661A6600F04E
:100050002CF8196E196E196E052000F02FF8012189
:100060000842F9D1002199601B49196000215960AB
:100070001A491B48016001219960EB211966A021F2
:10008000196600F012F800219960164914480160C1
:100090000121996001BC002800D000471248134993
:1000A000086003C880F30888084703B5996A0420EC
:1000B0000142FBD001200142F8D103BD02B5186610
:1000C0001866FFF7F2FF186E186E02BD00000240BE
:1000D000000000180000070000035F00212200005C
:1000E000F4000018222000A00001001008ED00E03C
:1000F00000000000000000000000000074B24E7A12
:1001000000200420F7010010CB010010CD010010E9
:10011000C9010010C9010010C9010010C901001077
:10012000C9010010C9010010C9010010CF01001061
:10013000C9010010C9010010D1010010D301001045
:10014000C1010010C1010010C1010010C101001067
:10015000C1010010C1010010C1010010C101001057
:10016000C1010010C1010010C1010010C101001047
:10017000C1010010C1010010C1010010C101001037
:10018000C1010010C1010010C1010010C101001027
:10019000C1010010C1010010C1010010C101001017
:1001A000C1010010C1010010C1010010C101001007
:1001B000C1010010C1010010C1010010C1010010F7
:1001C000EFF30580103800BE00BE00BE00BE00BECA
:1001D00000BE00BEF2EB8871F02400101425001060
:1001E0003802001090A31AE71E481F49086006C88D
:1001F00081F3088810471D480068002801D019487D
:10020000F3E70DA40ECC002902D000F012F8F9E7B4
:100210001749184A002000E001C19142FCD116495B
:100220008847164988471649884700BEFDE701C937
:1002300001C29A42FBD3704714250010C000002071
:10024000DC030020302800100000042000000420FF
:1002500030280010001004200010042000000000CE
:10026000704700000000000008ED00E0000000D032
:10027000DC030020700A0020B11C0010A90200104D
:10028000A91C0010F8B5C046044B10B5002B03D0D4
:100290000349044800E000BF10BDC0460000000054
:1002A00030090020A8230010F0B5DE464E46454632
:1002B0005746E0B51A2083B000F0BCF8D025802363
:1002C0002D06DB046B620620AB6100F0B3F8254C11
:1002D0000C22A4464023624491460126AB6201945D
:1002E000206800F0A7F8320008CC9A406A62AA6140
:1002F0004C45F5D11C4BD0269B46012300249A4641
:100300003606012001F056FE00220021062001F0F1
:10031000C5FE01F0F9FE53465C408023E4B2DB04E5
:10032000002C10D073610C235B445D469846012776
:100330003A0008CDFA209A40C000726100F004FC37
:100340004545F5D1DDE70127019DB3613A0008CDB0
:10035000FA209A40C000B26100F0F6FB4D45F5D19D
:10036000CFE7C046A8230010B4230010E12110B548
:100370004902074800F04CFD0221002000F00CF873
:100380000221012000F008F8024B1B7810BDC04686
:100390000040034010250010094A83009A1810B548
:1003A00014684022544080322240064CC000A446CB
:1003B00063441A60044B9C466044416010BDC046D3
:1003C00004C0014004D0014000400140C30810B502
:1003D000040007202040800081401800084C3C3079
:1003E000800001519B00002A04D0064A94466344D1
:1003F000196010BD044A944663441960F9E7C04689
:1004000000400140606101406071014080000029AE
:1004100005D0064B9C464023604403607047044B64
:100420009C46402360440360F8E7C04604E0014076
:1004300004F001400123D0228340120693629361AD
:10044000094A83009A1811684022514080320A40BC
:100450000649C0008C4663441A60054B9C46052340
:10046000604443607047C04604C0014004D001406E
:10047000004001400FB400B5084883B001F056FDBC
:10048000049B002B07D005A91800019101F0F2FB95
:10049000034801F04BFD012001F004FCC8230010CB
:1004A000D823001070B5EFF3108C72B60D4D2B6889
:1004B000002BFCD0BFF35F8F0724CB08C618C05CAD
:1004C00001230C40A3401C000440034207D1184301
:1004D0003070BFF35F8F2C608CF3108870BD1000FC
:1004E000FFF7C8FF2C0100D0044A1078431CDBB290
:1004F000172B00D9102313707047C04688030020C3
:100500000021044B044ABFF35F8F02C39342FAD128
:100510007047C046000100D0800100D0054B064A5C
:100520001360064A136053609360D3601361536194
:10053000936170478080808000E400E004E400E084
:100540001F2318401E3B8340002905D0C021044AC8
:100550004900535013607047802201498B50FAE7DD
:1005600000E100E070B50D00EFF3108672B60F4A9F
:100570001368002BFCD0BFF35F8F0D4B10309B68CE
:1005800084001B590B4A934203D09D4201D000F0D6
:1005900039FF074B9B681D51BFF35F8FBFF35F8F20
:1005A0000022024B1A6086F3108870BD240100D02F
:1005B00000ED00E0C1010010024B9C46614489003F
:1005C000016070474000003470B5114C114DAC42D1
:1005D0000FD2FF262368002B0CD0FFF785FF010008
:1005E0002000FFF7E9FFA680BFF35F8F0834AC421D
:1005F000F0D370BDFFF778FF01002000FFF7DCFFAC
:100600002671BFF35F8F0834AC42E3D3F1E7C046F5
:10061000D4030020DC0300200A4B1968EFF310809C
:1006200072B60A68002AFCD0BFF35F8F1B68BFF365
:100630005F8F00221A6080F3108840BF00200021E5
:100640007047C046640A0020F0B5DE4657464E4665
:100650004546E0B587B0EFF30583032201251A4034
:10066000954091008846A946B34B03925C58B34B22
:100670001D60B34B04934B46B24843630823E55EC9
:10068000002D37DAA3881BB2002B00DBADE0A37985
:10069000002B00D0EEE00823E05E002820DB4300C2
:1006A00062691B18DB00D3189E68DD68731C00D1DB
:1006B00011E1A44801004144826A0B69B71A9B1AF0
:1006C0009F4215D30123026A039883401A420FD038
:1006D0009C4800F047FB8D4202DCCCD18642CAD94F
:1006E00040BF07B0F0BCBB46B246A946A046F0BD2D
:1006F0000E61EDE762696B0092465B19DB009A447C
:1007000053469E68DF6800F02DFB8F42BADC00D1B3
:1007100003E1002F00DAE8E05246534652691B69B4
:100720009346049A934200D1D9E052460821605E74
:10073000528800045946104398470090019100994F
:10074000019A0B001000134300D1CEE013000A0001
:10075000B61A9F41002806DB7A4800F003FB009E92
:10076000019F36184F4153469E60DF6000229A5E1B
:10077000002A00DA86E7530099186069C900411819
:1007800002938B68C9689B46B94200DD7AE702D1C3
:10079000B34200D976E708239C46A44405956546F4
:1007A0002281A446029B2C0006E053009918C90040
:1007B00041188D68C968AB469B18DB00C318B94265
:1007C00006DC00D1B3E01C000023E25E002AECDA74
:1007D000230064469C4653461A806346059D1D804F
:1007E000A3881BB2002B00DA51E72269EFF31081D6
:1007F00072B61368002BFCD0BFF35F8F0123A7886C
:100800005B42A3803FB22369BFF35F8F00221A606F
:1008100081F31088002F00DA39E723000833220023
:100820009A4666697B00DB19DB00F318996850462D
:100830008C460824115FDD68002910DB029306E076
:10084000AB4244D00023E15E2000002906DB4C00CF
:100850006418E4003419E368AB42F1DD029B0780C1
:1008600000201F5E1980002FDCDA1400A379002B12
:1008700000D110E70023A37126000823E15E0836AB
:100880004B1C00D12CE70800A246656902E03E003F
:100890004B1C1AD04B005B18DB00EF180A008C468B
:1008A000E95E7B881BB2002BF1DA01235B42DC1787
:1008B000BB60FC60824205D0534631801B893B807F
:1008C00053461A8160464B1CE4D15446E5E6A368C2
:1008D0006345B7D9C2E76B1C00D0EAE6F8E65B4691
:1008E00058461B69984700281BD153461B8822692C
:1008F0002381EFF3108372B611680029FCD0BFF397
:100900005F8F514662880A8022696580BFF35F8FDE
:100910000021116083F31088B4E6864200D8F8E61F
:10092000B0E65B461A685B680092019307E7B3453F
:1009300000D848E74CE7C046480900203C70054015
:10094000490600100040054070B52E4C2569002D69
:1009500004D00A212C48FFF72FFE70BD2B4E032137
:10096000300000F0F5F9E660FFF7BEFD284B0322EA
:100970009C46D02322701B061B6801216370254B07
:100980006044A3600F2380002061022063806369BC
:100990004942A18019800231198647311D8358527E
:1009A00018315A5275325C399952183201319952C4
:1009B00018320131995218320131995208351832E2
:1009C0009D5202311832995218320131995218321F
:1009D000013199521832013199521832013199522C
:1009E0001832013199520C4B0C49DC6001303562F0
:1009F000FFF7B8FD01210320FFF7A2FD084B1D60A2
:100A0000A7E7C0468C030020640A00200040054090
:100A100040000034FFFF1000480900204906001084
:100A20003860054070B501000469EFF3108C72B6B0
:100A300020680028FCD0BFF35F8F02200D5E4C6958
:100A400068004019C00024180869002D36DB26888C
:100A50004E80BFF35F8F002606608CF31088E36042
:100A600063880498013320615B0405985B0CA260E5
:100A700060611A1C002B1FD093B2280462801843B7
:100A80000A69EFF3108C72B61368002BFCD0BFF329
:100A90005F8F8B8823808D800B69BFF35F8F00226F
:100AA0001A608CF310880B7801329A40CB680849A1
:100AB0008C4663441A6070BD0122DDE7BFF35F8F8F
:100AC000002303608CF3108801204042F3E7C04606
:100AD0003C20000010B543890A1493421ADD5300EC
:100AE0009B184269DB00D3180469EFF3108C72B6CF
:100AF0002268002AFCD0BFF35F8F5A88090494B2A1
:100B0000090C8A4208D00369BFF35F8F00221A6084
:100B10008CF31088002010BD8022120214435C80E8
:100B2000012302698371BFF35F8F002111608CF391
:100B30001088044902788C469340C26801206244C0
:100B40001360E8E73C200000F0B5C64600B582B06F
:100B5000040000F00FF9FA2206000F002000002325
:100B60000021920001F01CF88019794104000D1E4B
:100B700002DA01242E4D644206267642F717361912
:100B80006F41AF4214D811D000F0F4F832003B00AE
:100B9000121A8B41002B15DC002B46D020002900B7
:100BA00000F026F902B080BCB846F0BDA642EBD9F1
:100BB0000026002700F0DEF832003B00121A8B41BD
:100BC000002BE9DD00F0D6F832003B00121A8B4111
:100BD000002B0ADB00230193164B320000931648CA
:100BE0003B00FFF71FFF0130D8D000233900B0468B
:100BF0009C46124A1248536A994204D8966AB045F4
:100C0000CCD99942CAD10668EFF3108772B633681F
:100C1000002BFCD0BFF35F8F0368BFF35F8F664686
:100C20001E6087F3108820BFE5E7002AB6D0C9E729
:100C3000FFFFFF7F190600108C03002000400540D5
:100C4000640A0020F0B557464E46DE464546E0B5FC
:100C500006000F0085B0EFF3058399468B46002B05
:100C600012D0384900204B6ABB4206D38A6ADB1B8C
:100C7000591E8B41B2424041184305B0F0BCBB46FF
:100C8000B246A946A046F0BD2F4B9A46DB6898466F
:100C900053461B784046039300F064F84246039B9A
:100CA000040004339B009B580D001B1A39003000D0
:100CB000001BA941894510DC0DD020BF214A00202E
:100CC000536A5B45D9D3926ADB1B591E8B41B242F2
:100CD00040411843D1E78342EFD900F04BF832008E
:100CE0003B00121A8B41002B1ADB00230193174B98
:100CF0003200009350463B00FFF794FE011E0FDDCB
:100D0000104B5A6A5A451BD39B6AB34216D35046BE
:100D1000FFF7E0FE0B4A0020536A5B45ADD3D2E7F4
:100D2000084A0020536A5B45A7D30020926ADB1B68
:100D3000B24240415A1E934118439EE75A45E6D1BC
:100D400020BFE4E7004005408C0300201906001096
:100D500010B5024A0248FFF7A5FB10BDDC230010C6
:100D6000F80800200300416A0A00986A596A8A421A
:100D7000FAD17047034B596A0A00986A596A91423E
:100D8000FAD170470040054070B504000D00174AC5
:100D9000536A1900966A536A8B42FAD130001900DF
:100DA00024184D41AB4216D813D0104B2A005B6A71
:100DB0009D4203D90D494B6A9342FCD3934207D11C
:100DC0000A4A02E0516A994202D1916AA142F9D3DA
:100DD00070BDA642E9D9054B5B6A1C005A1CEFD0D6
:100DE000012201246442E5175242E3E70040054036
:100DF000064A536A9942FCD807D1044B02E05A6A6A
:100E0000914202D19A6A9042F9D870470040054059
:100E1000F8B5040006200D0000F02AFA002844D09E
:100E2000374B3849E3185A1E9341802212049446E6
:100E30005B429B0D344A9B0563441360334A136045
:100E400018000A689043FBD12D4B314AE3185942F0
:100E50004B4180215B0049000620995200F008FABE
:100E60002900C00000F0F8FB0130C3091ED1402763
:100E700001226262A362266BF30722D4E36A254B48
:100E80000620E51800232B60266300F0F1F93900F5
:100E9000800000F0E1FB7023E26A5A400E331340F9
:100EA0002B601D4B23630323A364F8BD1B4A9342AD
:100EB0001ED900231A4A1B4F6262A362266BF307F6
:100EC000DCD5194B144AE3181A60656AA36A062038
:100ED000AD01ED1800F0CCF9144900F0BDFBAD02F6
:100EE0000100280000F0B8FB0021FFF74DFFC5E727
:100EF0004006800E9F011A003F180300B9E7C04664
:100F00000080FCBF08C0004000E0004000F000404E
:100F1000680A00202C10000001030000FEFF000002
:100F2000FFFF0000C0FF3F00303000004E0E000009
:100F3000064A4300944680221B189B00634412011A
:100F40001A600022024B8000C250704700B000407F
:100F5000FC080020F8B5454657464E46DE46E0B54B
:100F60001E000A9B050088461700B34200D986E0A0
:100F70001A00330E994633029B46494600235846D1
:100F800000F0A8FB414B6C009C466419A4000200D1
:100F90006444002939D0636800234E469A462B1FCB
:100FA000DBB29946012B45D9C02380229B01E3186F
:100FB00012011A60364BAD0059599B46002907D0E3
:100FC000586900F049FB013043001B18033BFDD278
:100FD0007B01E027226853401F4080234A465B0183
:100FE000E3181F60012A3DD9802380229B01E3186A
:100FF00012011A60534663605B4601205E51F0BCEB
:10100000BB46B246A946A046F8BD802382469B0057
:10101000984236D300235846494600F05BFB060051
:1010200063689A45BBD9534663602B1FDBB2994670
:10103000012BB9D84346012BB6D1C02303229B0113
:10104000E3181A60023AA3681A42FCD07B01E02739
:101050002268AD0053401F4080230D4A5B01934638
:10106000E3181F6042462168514003220A401A607B
:10107000012243469A40A3681A42FCD0B4E70020FC
:10108000BDE780235B009A46CAE7C0460080004067
:10109000FC080020F8B5DE464E4657464546E0B50A
:1010A0008B4605000A991800160000F0D5FA0A9B35
:1010B0006C001F02324B64199C46A40064446368B0
:1010C00081469F4200D967602B1FDBB29846012BF7
:1010D00030D9C02380229B01E31812011A60294BEA
:1010E000AD0059599A4600291BD17301E0262268A8
:1010F00053401E40802342465B01E3181E60012AD4
:1011000030D9802380229B01E31812011A605346D4
:101110004A4667605A51F0BCBB46B246A946A04653
:10112000F8BD586900F098FA013043001B18033BE2
:10113000FDD2DAE75B46012BCBD1C02303229B0112
:10114000E3181A60023AA3681A42FCD07301E02641
:101150002268AD0053401E4080230A4A5B0192463C
:10116000E3181E605A462168514003220A401A6063
:1011700001225B469A40A3681A42FCD0C1E7C046F0
:1011800000800040FC080020F0B546464F46D64699
:10119000C0B51F00344B44009C462418A40064448E
:1011A000636888461600FF2B02D880235B006360CB
:1011B000031FDBB29A46012B30D9C02380229B014A
:1011C000E31812011A60294B8500595999460029E4
:1011D0001BD17301E026226853401E4080235246F3
:1011E0005B01E3181E60012A30D9802380229B0115
:1011F000E31812011A6080235B0063604B465F5165
:10120000E0BCBA46B146A846F0BD586900F024FAE1
:10121000013043001B18033BFDD2DAE74346012BA4
:10122000CBD1C02303229B01E3181A60023AA368C2
:101230001A42FCD07301E0262268850053401E400C
:1012400080230A4A5B019146E3181E6042462168EA
:10125000514003220A401A60012342469340A2688B
:101260001342FCD0C1E7C04600800040FC080020CB
:10127000014B8000C0587047FC080020F8B50400FE
:1012800021481E0017000D0000F0E6F901003800AB
:1012900000F0E2F9069B36041B031E432368002B73
:1012A00020DB1A4B1A49E3185A1E934180229201FF
:1012B00094465B421B0B174A1B0363441360164A98
:1012C00013601F000A689743FBD1144B2560E21896
:1012D0002123A06013602368002BFCDA0823E6605A
:1012E0001360F8BD3F2322681340AB42D9D1A368F5
:1012F0001B051B0D8342D4D1EE22E368D2021340BA
:10130000B342CED1EDE7C046001BB7000040FDBFA1
:1013100008C0004000E0004000F000400430000041
:101320002D2343607047C0468023024A9B000B4335
:10133000D362704700800540002310B50100988AF1
:101340001B8B984710BDC046162310B501001888A6
:1013500002331B88984710BDF8B54746CE4680B586
:101360000F1E18D0142399460433040000250126CB
:1013700098464B461888434621681B88984701C405
:10138000431E984101350640AF42F2D13000C0BC47
:10139000B946B046F8BD0126F8E7C046AA23064A7A
:1013A0001B0113602133FF33D3600449044B1960E0
:1013B0005368002BFCDA70470040024000B0FA008E
:1013C00000600240054A064B11681940054B0B436B
:1013D00013605368002BFCDB7047C046004002409E
:1013E000FF0F00FF00E0D100034A044B93605368F5
:1013F000002BFCDA7047C04600400240616D6F630D
:101400007047C04610B50148FFF734F800240010BB
:1014100070B5074D074EB54209D20024013E761B38
:10142000B60808CD984723000134B342F9D170BD06
:10143000602300109C230010054B064A06491A60E1
:10144000064A074B1A6010000B689843FBD170479F
:1014500000E00040BFCDFBFE08C00040FE7F3C0026
:1014600000F00040044BDB6C002B03D18022034BC7
:10147000D2021A607047C046000011504C20115033
:10148000044A054B1A60054A1368DB018033FBD11F
:101490007047C046FFFFFF0100F0004008C0004059
:1014A0004022034B9A675A671A67DA667047C0464C
:1014B00000F0014010B5FFF723F810BDF8B527493B
:1014C000274C284D641AA6103200302E00D9302245
:1014D0002800920000F0C0FBBC2C3BD830202F230A
:1014E0002C196407204A801BE40F9B1B052B16D97F
:1014F0003700002C02D0B300771CEA50001B3319D0
:101500009B004108EB18C900C9181A605A600833DB
:101510009942FAD1012303421CD09843C619B30063
:10152000EA50731C2F2E15D09B00EA50B31C2E2EB0
:1015300010D09B00EA50F31C2D2E0BD09B00EA50DC
:10154000331D2C2E06D09B00EA50731D2B2E01D08C
:101550009B00EA50054B9D60F8BDC046000100109D
:10156000C001001000000020C101001000ED00E0EB
:10157000002310B5294C82B0A367FFF70FFF0122AB
:10158000274B1A60636C012BFCD10322254B1A6098
:10159000224A936B012BFCD1013300930121224A93
:1015A00022480433FFF76AFE052301210093204AF5
:1015B0002048FFF763FE0022022104201E4BFFF7A4
:1015C000E3FD0022012105201C4BFFF7DDFD002279
:1015D000002107201A4BFFF7D7FD00220021082029
:1015E000174BFFF7D1FD8023DB0000930022002181
:1015F0000920134BFFF74EFD0022104B002106205F
:10160000FFF7C2FD0420FFF733FE0E4900F024F877
:1016100001000020FFF788FE02B010BD00800040EE
:101620003CB0004030B00040002F685900800240BC
:10163000008C864700C00240001BB700405973076A
:10164000006CDC0240420F0001480421014B1847A6
:10165000B003002059130010114A936F9B0813D256
:1016600010665166002905D0FFE7FFE7FFE7516FDD
:10167000106F704704B5002801D00020C04300F06F
:101680005FFE002104BDC046F0B5146E556E576F65
:10169000166FFFF7E5FF1466556657671667F0BDCE
:1016A000000000D094464A4A926F9208624601D2E6
:1016B00028E0C046F0B5464E346E756E776F366FD3
:1016C00000F020F89446424A14665566576716673C
:1016D0006246F0BD94463E4A926F9208624601D23D
:1016E00054E0C046F0B53A4E346E756E776F366F83
:1016F00000F04CF89446364A1466556657671667EC
:101700006246F0BD002B24DB11D000293EDA00B583
:10171000C943404200D1013100F038F8C94340428A
:1017200000D10131DB43524200D1013300BD002A18
:10173000EBD1002801D1002905D00020C90FC9072D
:1017400001D1C043410800B500F0F2FD00220023A2
:1017500000BD00B500290ADBDB43524200D1013352
:1017600000F014F8C943404200D1013100BDC94323
:10177000404200D10131DB43524200D1013300F03D
:1017800005F8DB43524200D1013300BD002923D1CB
:10179000002B18D1002A0CD0BC460D4F38667A6653
:1017A00000210023FFE7FFE7FFE77A6F386F674606
:1017B0007047002801D00748010000B500F0B8FDCF
:1017C0000022002300BD02000B0000200021704712
:1017D000000000D0FFFFFFFF002B00D0BFE0130C84
:1017E00028D1002AE7D080B4114F39667A66FFE726
:1017F000FFE730B4040C7B6F396F1B0423433B6657
:101800007A66FFE7FFE7FFE7C04684B27B6F3D6F74
:101810001B0423433B667A66FFE7FFE7C0460023CD
:101820002C042D0C7A6F386F00196941B0BC7047D9
:10183000000000D0F0B594460025140E01D112022C
:101840000835140F01D112010435940F01D1920013
:101850000235D40F01D152000135D40B0134254F8C
:101860007C66254C3C660E0C93B2FFE7FFE7FFE772
:101870003C6F6643360C7703BE467343DF0B5B0455
:10188000C01AB941130C7343DB18C91ACE0866435A
:10189000360CB64493B273431F0F1B01C01AB941F3
:1018A000130C73431F0B1B05C01AB941860D8F0221
:1018B0003E436643360C092D24DB520A7243801ADC
:1018C0007703460A6643360C16235B1BDE40DF4077
:1018D000BF1964466643821B704604350633010017
:1018E000D940A840C01900D30131A24206D200233A
:1018F000F0BD0000000000D0FFFFFFFF121B013011
:10190000F3D3F1E709277F1BFE406446A2B272437E
:10191000801A00D20139220C7243130C1204821A6D
:1019200099410B007046043513370100F940A84077
:10193000801900D30131002B02D1A2420AD2F0BD9E
:10194000013000D30131121BFAD2013BF8D1A2427F
:1019500000D2F0BD013000D30131121BF7E7F0B522
:101960001C0C00D080E00CB400251C0A04D11B0222
:10197000160E3343120208351C0B04D11B01160F3F
:101980003343120104359C0B04D19B00960F334363
:1019900092000235DC0B02D192185B4101351C002C
:1019A000971864410134464F7C66464C3C660E0CE9
:1019B000FFE7FFE7FFE7C0463C6F6643360C77035F
:1019C000BE4697B27743C01B00D20139C01B00D27C
:1019D00001399FB27743C91BC91B170C77437E049B
:1019E000FF0B801BB941CE086643360C0C2D33DB50
:1019F000B644120B1F053A431B0B97B27743C01B2B
:101A000000D201399FB27743C91B170C77433E04BC
:101A10003F0C801BB941860D8F023E436643292748
:101A20007F1BFE400C3D7746AF40BF1930BCA2B2D1
:101A3000ABB272437343801A9941220C7243130C68
:101A40001204801A994102000B000137001BA941C2
:101A5000F9D2781E0021F0BD0C277F1BFE4077468F
:101A60007F0BAF40FF19E0E700245D1C07D0144F47
:101A70007D663966FFE7FFE7FFE7FFE73C6F95B25A
:101A80009EB265436643401BB141150C1E0C654375
:101A9000664336042F0C3E432D04401BB14199424E
:101AA00004D202000B0020000021F0BD01D19042C1
:101AB000F7D3801A994101349942F2D3F6E7000036
:101AC000000000D0FFFFFFFF10B50148FEF7D2FC79
:101AD0000C240010132370B51D78012D19D014DDCE
:101AE0001D48FFF731FC06001C48FFF72DFC1C4C7D
:101AF00080223100200000F0AFF8022D06D01948F6
:101B0000FFF71AFC184B186070BD154C174BA364F7
:101B1000F5E7174B124C23606360A360E360236119
:101B20006361A361E36123626362A362E36223638F
:101B30006363A363E36323646364A364E36423656F
:101B40006365A365E36523666366A366E36623674F
:101B50006367A367E367D9E7534400005346000077
:101B6000600500204C33000060090020751B001048
:101B7000C91A001007B5604601880A0A0230DF2A38
:101B8000FAD1C9B2820804D3028840880004104305
:101B900000E00068014A5050039007BD6005002036
:101BA00051434343C9188C46110C83B24B4310B4C4
:101BB000040C614392B280B2504362431C041B0C7C
:101BC000001910BC59411304120CC0185141614452
:101BD0007047000010B50148FEF74CFC24240010AB
:101BE000132310B510481C78FFF7AEFB0100012C41
:101BF0000AD003DD80220D4800F02EF80C48FFF7D4
:101C00009BFB0C4B186010BD084C5422200000F0C8
:101C100023F82200084980322368002B00D121607C
:101C200004349442F8D1E9E75346000064090020E7
:101C30004C33000060090020D51B0010014804212E
:101C4000014B1847C003002059130010014B1B68BB
:101C500018470000C0030020014B5B6818470000D4
:101C6000C003002010B5002800D110BD00F014F909
:101C7000FBE7C04610B5094A0300146884B0002C85
:101C800008D0012200910648524203A9A047012032
:101C900004B010BD00F04AF90020F9E72C0900203B
:101CA000651C001000BEFDE710B5FFF7FBFFC04646
:101CB00070B5FFF7ADFB074D074EB54209D20024C2
:101CC000013E761BB60808CD984723000134B34285
:101CD000F9D170BD9C230010A8230010030010B59B
:101CE000080011001B68984710BDC046F0B5C646F5
:101CF00000B5437D07000C001600002B46D0002ADB
:101D000017DD0B780A2B24D000239846012E13D020
:101D100001252900635C01350A2B26D0B542F8D194
:101D2000464509DCA419013C23780D3B5A42534136
:101D30003B7580BCB846F0BD4346E018A419F11AC3
:101D4000013C3B68984723780D3B5A4253413B7511
:101D5000EFE7037D002BD7D102210F483B6898475E
:101D6000012EDFD001239846D2E7631E5B5C0D2B6A
:101D7000D4D0884504DA4346C91AE0183B6898472E
:101D8000022105483B68A8469847C7E70368110049
:101D900020009847CDE7C046EC240010F0B545463A
:101DA000DE464E465746E0B583B091461C0080465D
:101DB0000D00FEF7DFFF0023304A12184B41002BC5
:101DC00002DA01222E4B52422E4908008A4600F0C8
:101DD000BFFA07006B1C03D1404600F007FA05006C
:101DE000002C27D0284E294B1C68002C18D04B46BD
:101DF000002B21D1264B994602E02469002C0FD0FC
:101E00002368002BF9D04B461B68002B01D09C4265
:101E1000F3D120002A004146B0472469002CEFD1BD
:101E2000002F26D1280003B0F0BCBB46B246A9461D
:101E3000A046F0BD174ED6E7154B99460A239B46A0
:101E400002E02469002CEBD02368002BF9D04B462C
:101E50001B68002B01D0A342F3D12A004146200089
:101E6000B0476B465A462000DA71D91D0122B047AF
:101E7000E7E7504600F054FAD4E7C04640420F006E
:101E8000FFFFFF7FD4030020ED1C00102409002079
:101E900028090020DD1C0010F0B5CE46474680B56D
:101EA00083B06B460600DD1D2870FEF763FF00233C
:101EB000194A12184B41002B02DA0122174B5242E9
:101EC00017490800884600F043FA164B81461C6803
:101ED000002C14D0144F02E02469002C0FD023688A
:101EE000002BF9D03B68002B01D09C42F4D120009C
:101EF00001222900FFF7FAFE2469002CEFD14B469E
:101F0000002B05D1300003B0C0BCB946B046F0BDCF
:101F1000404600F005FAF5E740420F00FFFFFF7F63
:101F2000D4030020240900202809002070B50400F3
:101F300000F05CF901230100050001222000FFF7F9
:101F40002DFF084B1C68002C06D06368002B05D0C1
:101F500098472469002CF8D1280070BD2469002C12
:101F6000F3D1F9E72409002010B5024800F004F885
:101F700010BDC0465809002010B588B004000D22DD
:101F800000216846FFF762FE0D22002104A8FFF73A
:101F90005DFE4B236A466846137004A90D2200F0CB
:101FA000B7F91521082220006944FFF755FE08B053
:101FB00010BDC04610B5334B82B01870012834D024
:101FC00002282FD1304C002223000021042000944D
:101FD000FEF7C0FF23000022002105200094FEF739
:101FE000B9FF0820FEF7A4FF0720FEF7A1FF274B4B
:101FF00002220021009309202300FEF7ABFF2300FB
:102000000022002106200094FEF7A4FF2048FFF7DD
:1020100087F92048FFF784F9FFF7D4F9FEF7A6F90E
:1020200002B010BDFFF7EEF9CCE71B4C00222300F5
:10203000022100940420FEF78DFF230000220021DE
:1020400000940520FEF786FF0820FEF771FF0720A9
:10205000FEF76EFF0D4B03220093002123000920A1
:10206000FEF778FF23000022002100940620FEF7EF
:1020700071FF0748FFF754F90648FFF751F900F0E0
:1020800057F8CBE76C0A0020A02E63001BB70000B6
:102090000080024000C00240001BB70070B5040081
:1020A000002926D1012302255A40AD1A2000FEF74F
:1020B000C1F901212000FEF7A9F901222900200021
:1020C000FEF784F90E4B1B78012B0FD000F048F877
:1020D0000722224092009540E3080A4A3C339B00C5
:1020E0009D5000212000FEF791F970BDFFF77CF9AB
:1020F000EEE753425A41032355429D430835D5E745
:102100006C0A00200040014010B500F03DF8A82204
:10211000064B9958012149429950043298589950D8
:10212000FFF726FAFEF722F910BDC04600800040F6
:102130008020074A074B116840041940064B0B43A7
:102140000649086013609369002BFCDB7047C046AA
:1021500000000640FF0F00FF00E0D10018300640ED
:102160008022054B52041A60044A054B1A60054A46
:102170009369002BFCDA704718300640616D6F637D
:102180000C000640000006408022054B52041A60F5
:10219000044A054B13609369002BFCDA7047C04674
:1021A000183006400000064000F0FF0010B50100A6
:1021B00000230022002000F047F810BD70B5074C46
:1021C000074D641BA41005D0013CA300EB589847B1
:1021D000002CF9D100F098F870BDC046A82300107B
:1021E000A82300107047C0467047C04610B583074B
:1021F0000AD00300032102E001330B4205D01A7814
:10220000002AF9D1181A10BD030019680C4A0D4CA8
:102210008A188A4322420FD15968094A04338A181E
:102220008A43224208D15968054A04338A188A43EE
:102230002242F1D000E001331A78002AFBD1E1E715
:10224000FFFEFEFE80808080F0B5D6464F464646B3
:102250009846244BC0B5060018689A460F00914670
:10226000FFF7C0FF204B1D68002D32D053466C682D
:1022700018681F2C30DC002E0CD1631C0234A40023
:102280006B606751FFF7B0FF0020E0BCBA46B14673
:10229000A846F0BD49468822A300EB189950C421F6
:1022A00049008C46AC446146873AA2400968914691
:1022B0001143624611608421424649005A50022E61
:1022C000DBD129004A468D31FF310B6813430B6087
:1022D000D3E7064D1D60C9E7FFF786FF01204042A6
:1022E000D3E7C046D003002060060020640600202B
:1022F000034B10B5002B02D00248FFF757FF10BD6B
:1023000000000000BD210010F8B5C046000000002C
:1023100001B40248844601BC604700BF350200207A
:1023200001B40248844601BC604700BF5901002047
:1023300001B40248844601BC604700BF710300201D
:1023400001B40248844601BC604700BF710300200D
:1023500001B40248844601BC604700BFC1000020B0
:102360003914001065140010491600103D1C0010AF
:10237000D51A0010E11B0010711500108114001017
:10238000A1140010B5140010C9050010BD140010F0
:1023900049090010011400101D050010F122001061
:0823A000691F00108902001002
:1023A8001D0000001C0000001B0000001B000000B6
:1023B8001C0000001D0000000800525092000000A0
:1023C8000A2A2A2A2050414E4943202A2A2A0A004A
:1023D8000A000000486172647761726520616C616F
:1023E800726D20256420616C726561647920636C6C
:1023F80061696D65640000004861726420617373EF
:10240800657274006D697373696E6720646F7562B5
:102418006C652066756E6374696F6E00000000005D
:1024280052656C6561736500626F6F74325F7732F5
:102438003571303830000000302E3100322E322E07
:102448003000000073656565645F7869616F5F726D
:102458007032303430000000706F7765722D73650C
:10246800712D736F6674776172652D736565656428
:102478002D72703230343000536570202034203291
:102488003032350006005250D3F07542282400102F
:1024980006005250E182887F302400100600525016
:1024A8003ABCA9114024001006005250ABB3605347
:1024B8004424001006005250BBFF3CB64C240010C8
:1024C80006005250861C0302602400100600525079
:1024D8005422A29D8024001005005250DE65F46845
:0824E800302800100D0A00006D
:1024F0008C24001098240010A4240010B024001094
:10250000BC240010C8240010D4240010E0240010C3
:04251000C0230010D4
:10251400F0B5C646150000B504001E000268EFF3CE
:10252400108172B61368002BFCD0BFF35F8F0423B5
:10253400E3562268002B2BDBBFF35F8F0020106073
:1025440081F31088D02212061278002752B29046E6
:102554009A420ED1002080BCB846F0BDBFF35F8F15
:10256400176081F310882800310000F02DF900284D
:10257400F0D12268EFF3108172B61368002BFCD0FF
:10258400BFF35F8F237922687F2BE7D9434602E0AC
:10259400D0231B061B682371BFF35F8F00231360D6
:1025A40081F310880120D6E70268EFF3108172B638
:1025B4001368002BFCD0BFF35F8FFF230371036804
:1025C400BFF35F8F00221A6081F3108840BF704709
:1025D40010B5084C2378002B0AD1802306480749FC
:1025E4005B051A68C25004338B42FAD1012323706D
:1025F40010BDC0466D0A0020F8070010000100104D
:1026040010B5014B984710BDF9070020064B5A68D6
:1026140002609A684260DA6882601A69C2605A6924
:1026240002619B6943617047000002400268064BE7
:102634005A6042689A608268DA60C2681A61026904
:102644005A6142699A61704700000240034B1A685C
:10265400C0239B009343024A136070470C800140DF
:102664000C900140054B1A6880239B005340C02204
:1026740092001340024A13607047C0460C80014028
:102684000C9001400023F0B5DE4657464E464546C1
:102694009A46E0B589B001900E00988A45491B8B93
:1026A40014009847534681464349988A1B8B9847A0
:1026B400534642490500988A1B8B98478046FFF78A
:1026C40087FF02A8FFF7A2FFC847A847FFF7CAFF82
:1026D400251E22D00823C0219C46022049056246BB
:1026E4008B6A1A4018423FD0631B002D2FD1002A59
:1026F40011D1002C11D0C0235B059B4602239A46BE
:10270400063399465B464A4657469B6A1A401F421F
:1027140042D0002AF6D0002C30D1FFF797FFC047F3
:10272400FFF76EFF02A8FFF781FF09B0F0BCBB46BC
:10273400B246A946A046F0BD002C2FD1C0225205B6
:10274400926A914608224F463A40BF072DD50D2B79
:102754001BD9002AF0D1C0225205926A9146082260
:102764004F463A40BF07F2D4002A04D12B0023433A
:10277400002BB4D1D1E72B00002CF9D00B6E013C17
:102784003370230001362B43F2E7019F013D3B7870
:1027940001370B660197E7E70025E5E7C0235B05F2
:1027A4001B6E013C3370013699E72B00002ADFD100
:1027B400DCE7C04649460000455800004643000097
:1027C4007047C0460000000001B40248844601BCC2
:1027D400604700BF450C001010000000000000001E
:1027E40000000000000000000000000000000000E5
:1027F400E0030020000000000000000000000000D2
:10280400503300004C3300005433000052330000B6
:102814004D5300004D430000533400004334000086
:0C282400F407002000000000000000008D
:04000005100001E9FD
:00000001FF
